:100000000C94DB070C9403080C9403080C9403086D
:100010000C9403080C9403080C9403080C94030834
:100020000C9403080C9403080C94580B0C94CA0B02
:100030000C9403080C9403080C9403080C94030814
:100040000C9403080C9403080C9403080C94030804
:100050000C9403080C9403080C9403080C948B0E66
:100060000C9403080C9403080C9403080C940308E4
:100070000C9403080C9403080C9403080C940308D4
:100080000C9403080C9403080C9403080C940308C4
:100090000C9403080C9403080C9403080C940308B4
:1000A0000C9403080C9403080C940308F0F89C8E3D
:1000B0008783878E9CF8F00000FEFF030303030391
:1000C000070EFCF80000FEFF0303030303070EFC0A
:1000D000F80000FFFF00000000000000FFFF00002C
:1000E000FEFF8383838383C7EE7C380000F8FC0E19
:1000F00007030303070EFCF800003F7FE0C0808089
:10010000C0E07F3FFFFF01010101010101FFFF008E
:1001100000FFFF0C0C0C0C1C3E77E3C100007FFFBE
:10012000C0C0C0C0C0E0703F1F00001F3F70E0C0F3
:10013000C0C0E0703F1F00007FFFC1C1C1C1C1E36B
:10014000773E1C00001F3F70E0C0C0C0E0703F1F42
:10015000000000000001FFFF01000000D5F08D1439
:10016000A1C881CFD9F1AF20007374617465476174
:100170006D654F76657200596F75206172652069F3
:100180006E207468650050726573732041202D3EA7
:10019000204D656E75496E74726F0000000000009E
:1001A000000000B0480848E85020000000000000AF
:1001B000000000000040406020BCBA65C90F1AC8AA
:1001C000C911784040408000000000003C66C3999F
:1001D000CF7526F3FCBF782F033D64C69DC3663CF4
:1001E00000000000000000000000006090109090EF
:1001F000A0C000000000000000000080C0A020207F
:10020000F09E61A3455B9232AA27E9720C0C0000B4
:10021000000000070F1115151E04021D3C3C2C0F99
:100220000303023F5B85FD7A000000C02EF961499F
:10023000194AC47020209824F098881830E00000F3
:1002400000000002050B86EE77E949A25C8A5A316C
:100250000306040603010000000000000403013C43
:1002600065C691CE663C0000000000000000000062
:10027000000000000000000000E01068A838D4D2A0
:1002800042523254480000000000003C66C399D33B
:100290005539DB1421CE21EA12FC50988800000069
:1002A00000000000000000000000000103003C67A7
:1002B000C99BC3663D00000000000078CC8612F6A2
:1002C000CC780040C0C000000080808000000000AA
:1002D0000000000002251D3F6A5AE71A23C41B28AC
:1002E000DF654461331E000000000000000024545C
:1002F000DC9485967018130E0101010100000000C6
:1003000000000000000000000000000000000000ED
:1003100000000000000000000000000000000000DD
:10032000000000001078AC740464B8000000000005
:100330000000000F1F1A0B0BCDFF8FF93929331363
:100340007F513F000000000000000000000000009E
:10035000000000000000000000000000000000009D
:1003600000000040C0C0C004FC1CDCF880E0A09C81
:100370006242FA5ED46838E0C0000078EFE6F7F633
:10038000FFEC7D0F3A7A7A7E0374FCE5F17E3F0F35
:100390000100000000000000000000B0580848E81C
:1003A00050200000000000000000000000404060FD
:1003B00020BCBA65C90F0AD839E1F8404040800036
:1003C000000000003C66C399CD773A0F3C317C2F8A
:1003D000033C67CF99C3663C0000000000000000AA
:1003E00000B864842474A89000000000000000009D
:1003F0000000000000404040FE5D12A44586769655
:10040000C49EE8C82860C080000000003C66C38924
:10041000CB6E36030E12170800070E1913180C07BF
:10042000000000C0AE59A189D92AA480D020A058CC
:10043000EC7058C81830E0000000000106192C28A4
:10044000C9E57034E093849F61430604060301000C
:100450000000000000000407003C64C281DF663C2D
:10046000000000000000000000000080C06020606C
:10047000C090A06010E828B854524252325448004C
:10048000000000070C18161C040F18FF1019A672A4
:100490004DF678C48000000000000000000000005D
:1004A0000000000001033C66C39FC3663C000000DF
:1004B00000000078CC8672C6CC7880E87C4858E092
:1004C000785C963286CC78000000000000050505B7
:1004D0003F13374FBC6186CD3A8A75B575F0E0E0C1
:1004E00070000000000024549C9486927308080B4E
:1004F00006010100000000000000000000000000F4
:1005000000000000000000000000000000000000EB
:10051000000000849A29FB61492ED0C82870600031
:100520000000000000000000000000010305030EB1
:1005300034E0A0ED5B0400000000000000000000BB
:10054000000000000000000000000000C02020208B
:1005500020C000000000000000000000C06040401B
:100560007CCA91AB345162766EA683E0F058E89075
:100570000000003C766361697B3E366F7F2D353924
:100580001F137FC3E6783F0F00000000000000004B
:100590000000B0480848E8502000000000000000BB
:1005A00000000000000000003C7AE5DF3F7260615F
:1005B00041E00000000000000000000078C58393C7
:1005C000DB4D273C3D703F0F74CB8D9B854A30003F
:1005D000000000000000DC724292BAD44800C00063
:1005E00000800000000000000000000080808FF606
:1005F0005CD212A283F5281B75DD963286CC78007A
:10060000000000003C66C297DC6639030404050262
:100610000000010101000000000000C02EF961C9C6
:10062000D92AA480F880F8CCA63286CC78000000C5
:1006300000000007182F4A5756562E2BE3F44CB7EC
:10064000CD3509000000000000000000000000009F
:10065000000000003F033E60C29DC3663C000000F6
:10066000000000F0980CE48CD8305C902CE41CAABC
:10067000692109392A240000000000000103020357
:1006800073CE2E3124635DE2CE70200000000000A6
:10069000000000000000000000003C66C399CF6726
:1006A0003C03040000000000000000000000000007
:1006B0000000804080FCF65B898366BC800000807F
:1006C00000000078CC8632E64CFB921CE30812A1B5
:1006D000AED72351A84E7F0F000000000001010596
:1006E0000223559A968595547850292F191E00009B
:1006F00000000000000000000000000000000000FA
:100700000000000000000000000000041A697BE106
:10071000DB2EC00000000000000000000000000010
:10072000000000C0FBCF790A172E31221F0E1C00DB
:1007300000000000000000000000008080808000B9
:1007400000000000808080B8E44464E4A8900000C9
:10075000000000000F0B556AD4CC4A458292A29645
:100760004526E8B8C04040C0000000001C36636960
:100770006D6A3639787C5C1D1F013F73636F61734E
:100780003E0000000000000000008070A8A80828BB
:1007900070B08080000000000000000080C0406059
:1007A000FE81B8A3224615FDC59EE261E04000002F
:1007B0000000000079CF8392CC7C020D1E33111F04
:1007C000011F3123180F000000000000C02EF96146
:1007D000C999AAA440808040A08080000000000049
:1007E00000000000CF57E92A0AD115063A489D3784
:1007F000654C61331E000000000000013C66C39A96
:10080000CA673F0102020101000000000000000071
:100810000000000000000000C02050B05C92425276
:100820003254480000000000000000E03019CBBA4C
:10083000E729FA235418CB340CF0704880000000EC
:100840000000000103060406030001060605013D41
:1008500067DF91C3663C000000000000000000005C
:100860000000000000000000000000000000000088
:100870000000000000000000000000000000000078
:100880000000000000000000000000000000000068
:100890000000000000000000000000000000000058
:1008A0000000003C66DB79C3661C30C0F80000C461
:1008B0003C3CFC0000000000000000000088BC83FD
:1008C00062B32D410BD4745750E72438E810E00090
:1008D0000000001E33614C6D371D02011F012564AD
:1008E0009D9784947F040300000000000000000036
:1008F00000000000000000000000000000000000F8
:1009000000000000000000000000000000000000E7
:100910000000C020E06020E0C0000078ECE4E4E4E7
:10092000E2E473033A7A7A7E0975FEE5F17E3F0FC1
:1009300001000058D4B46CACE8104FBE8670202083
:1009400038A4B098881830E00000000F3B50A32472
:100950001299C72508E29D8D5B300006040603014D
:100960000000000000000403013C67C291DF663C08
:100970000000000000000000000000737461746556
:100980004D656E75506C617900596F7520617265A7
:1009900020696E2074686500507265737320412071
:1009A0002D3E2047616D65506C6179696E670073FB
:1009B000746174654D656E7548656C7000596F752E
:1009C0002061726520696E207468650050726573DD
:1009D000732041202D3E204D656E75506C6179006D
:1009E0004C657427732052696465004172647562B6
:1009F000696B65005072657373204120746F2050DD
:100A00006C61790073746174654D656E75496E74BF
:100A1000726F00596F752061726520696E2074686D
:100A2000650050726573732041202D3E204D656E28
:100A3000754D61696E00080B000202020100090495
:100A4000000001020200000524001001052401013C
:100A50000104240206052406000107058103100095
:100A60004009040100020A000000070502024000DC
:100A7000000705830240000004030904120100027C
:100A8000EF0201404123368000010102030141725F
:100A90006475696E6F204C4C430041726475696ED9
:100AA0006F204C656F6E6172646F00000000000083
:100AB0003E5B4F5B3E3E6B4F6B3E1C3E7C3E1C18CC
:100AC0003C7E3C181C577D571C1C5E7F5E1C00182A
:100AD0003C1800FFE7C3E7FF0018241800FFE7DB1E
:100AE000E7FF30483A060E2629792926407F05057A
:100AF00007407F05253F5A3CE73C5A7F3E1C1C08B7
:100B0000081C1C3E7F14227F22145F5F005F5F067B
:100B1000097F017F006689956A606060606094A2C9
:100B2000FFA29408047E040810207E201008082AE2
:100B30001C08081C2A08081E101010100C1E0C1E81
:100B40000C30383E3830060E3E0E06000000000025
:100B500000005F00000007000700147F147F1424CA
:100B60002A7F2A122313086462364956205000084F
:100B7000070300001C2241000041221C002A1C7FA8
:100B80001C2A08083E080800807030000808080881
:100B900008000060600020100804023E5149453EF4
:100BA00000427F400072494949462141494D33186E
:100BB00014127F1027454545393C4A4949314121A6
:100BC0001109073649494936464949291E0000148A
:100BD00000000040340000000814224114141414D2
:100BE00014004122140802015909063E415D594E84
:100BF0007C1211127C7F494949363E414141227F96
:100C00004141413E7F494949417F090909013E412E
:100C10004151737F0808087F00417F410020404117
:100C20003F017F081422417F404040407F021C0268
:100C30007F7F0408107F3E4141413E7F090909063C
:100C40003E4151215E7F091929462649494932030F
:100C5000017F01033F4040403F1F2040201F3F4095
:100C600038403F631408146303047804036159494E
:100C70004D43007F414141020408102000414141A1
:100C80007F04020102044040404040000307080086
:100C900020545478407F2844443838444444283809
:100CA0004444287F385454541800087E090218A47C
:100CB000A49C787F0804047800447D4000204040D4
:100CC0003D007F1028440000417F40007C047804F0
:100CD000787C080404783844444438FC18242418E8
:100CE00018242418FC7C0804040848545454240490
:100CF000043F44243C4040207C1C2040201C3C40BD
:100D000030403C44281028444C9090907C446454DB
:100D10004C440008364100000077000000413608CE
:100D20000002010204023C2623263C1EA1A16112FE
:100D30003A4040207A38545455592155557941212B
:100D400054547841215554784020545579400C1E14
:100D500052721239555555593954545459395554BC
:100D600054580000457C410002457D420001457C0D
:100D700040F0292429F0F0282528F07C545545001E
:100D80002054547C547C0A097F4932494949323203
:100D900048484832324A4848303A4141217A3A423A
:100DA000402078009DA0A07D39444444393D404016
:100DB000403D3C24FF2424487E4943662B2FFC2FD2
:100DC0002BFF0929F620C0887E090320545479415D
:100DD0000000447D413048484A32384040227A0081
:100DE0007A0A0A727D0D19317D2629292F28262994
:100DF00029292630484D40203808080808080808E6
:100E000008382F10C8ACBA2F102834FA00007B0025
:100E10000008142A142222142A140895002200958E
:100E2000AA005500AAAA55AA55AA000000FF001062
:100E30001010FF00141414FF001010FF00FF10101A
:100E4000F010F0141414FC001414F700FF0000FF5D
:100E500000FF1414F404FC141417101F10101F10BA
:100E60001F1414141F00101010F0000000001F10B9
:100E70001010101F10101010F010000000FF1010C4
:100E800010101010101010FF10000000FF140000D0
:100E9000FF00FF00001F10170000FC04F4141417DB
:100EA00010171414F404F40000FF00F714141414C1
:100EB000141414F700F7141414171410101F101F33
:100EC000141414F4141010F010F000001F101F0080
:100ED00000001F14000000FC140000F010F01010BF
:100EE000FF10FF141414FF141010101F0000000056
:100EF000F010FFFFFFFFFFF0F0F0F0F0FFFFFF004A
:100F000000000000FFFF0F0F0F0F0F38444438445C
:100F10007C2A2A3E147E02020606027E027E0263BC
:100F2000554941633844443C04407E201E2006025B
:100F30007E020299A5E7A5991C2A492A1C4C720138
:100F4000724C304A4D4D303048784830BC625A4679
:100F50003D3E494949007E0101017E2A2A2A2A2A6A
:100F600044445F444440514A444040444A51400054
:100F700000FF0103E080FF000008086B6B083612D9
:100F8000362436060F090F0600001818000000105E
:100F900010003040FF0101001F01011E00191D1744
:100FA00012003C3C3C3C0000000000010204081020
:100FB00020408000561411241FBECFEFDAE0DEBFC0
:100FC000CDBF11E0A0E0B1E0E2E2FAE202C005909C
:100FD0000D92A034B107D9F725E0A0E4B1E001C03B
:100FE0001D92AA3CB207E1F717E0CBEDD7E004C0B1
:100FF0002197FE010E940415CA3DD107C9F70E943E
:101000004B100C940F150C940000FC0180915001C2
:10101000811103C08FEF9FEF08959FB7F89482E08E
:101020008093E9002091F20030E01216130614F4C8
:1010300021E030E02115310559F0289884E68093AD
:101040004F018091F10080838091F200882319F094
:101050009FBFC90108958BE68093E800F9CF2FB7B1
:10106000F89483E08093E9009091E800892F8072E2
:1010700095FF04C09091F20080E4891B2FBF089572
:1010800080916D0581110DC082E08093690584E037
:1010900080936A0510926C0510926B0581E0809335
:1010A0006D0589E695E00895CF93DF931F92CDB744
:1010B000DEB76983DC01ED91FC910280F381E02DC4
:1010C00041E050E0BE016F5F7F4F09950F90DF91C7
:1010D000CF91089583E08093E9008091F200882306
:1010E00019F08AE38093E80008950E942F0890E0A9
:1010F0000895CF93DF931F92CDB7DEB7FC018485AF
:10110000958597FD05C02FEF3FEF358724870BC0EE
:10111000CE0101960E940508019719F4898190E09B
:1011200002C08FEF9FEF0F90DF91CF9108950F9343
:101130001F93CF93DF931F92CDB7DEB78C01FC01D5
:101140008485958597FF0EC0CE0101960E94050803
:10115000019719F4298130E002C02FEF3FEFF80129
:1011600035872487F801848595850F90DF91CF918D
:101170001F910F910895FC018485958597FD0BC003
:101180009FB7F89482E08093E9008091F2009FBFBE
:1011900090E0019608959FB7F89482E08093E9006B
:1011A0008091F2009FBF90E008958F929F92AF923E
:1011B000BF92CF92DF92EF92FF920F931F93CF9344
:1011C000DF935C016B017A0180911101882309F49E
:1011D0005BC080915001882309F456C080914E0174
:1011E00080FF05C08091E00082608093E000E7010D
:1011F00010E00AEF83E0882E9AE3992E2097D9F128
:101200000E942F0881110AC0015009F43DC061E01D
:1012100070E080E090E00E94510EF0CF282F30E087
:10122000C217D3070CF48C2F4FB7F8948092E900C3
:101230009091E80095FF1DC0282F30E0C21BD30B12
:10124000F601982F915020F081918093F100FACF10
:10125000C20ED31E112319F09092E80009C08091AC
:10126000E80085FD06C09092E80011E0209709F0A3
:1012700010E04FBFC3CF1111C3CF5D9884E68093B8
:1012800068051E141F0444F081E090E0F50193838B
:10129000828380E090E001C0C701DF91CF911F9170
:1012A0000F91FF90EF90DF90CF90BF90AF909F9005
:1012B0008F9008950F931F93CF93DF931F92CDB715
:1012C000DEB782E0898342E450E066E37AE080E8BA
:1012D0000E9417100E944008DC0112960D911C918B
:1012E00013970115110569F0D801ED91FC91028069
:1012F000F381E02DBE016F5F7F4FC801099597FF15
:1013000007C089810F90DF91CF911F910F910895B0
:10131000F80100851185E5CF20915B05282329F48C
:1013200090915A05982381E009F480E008950F9385
:101330001F93CF93DF938C01C0E0D0E0F801EC0F56
:10134000FD1F6491662371F0E0915105F091520503
:101350000190F081E02D81E595E00995892B11F050
:101360002196ECCFCE01DF91CF911F910F9108957F
:10137000E1E5F1E0A0E0B8E000800EBC8111012CB5
:101380001197A0FDFDCF0192B9F70DB408952F92EA
:101390003F924F925F926F927F928F929F92AF9205
:1013A000BF92CF92DF92EF92FF920F931F93CF9352
:1013B000DF93CDB7DEB728970FB6F894DEBF0FBE28
:1013C000CDBF5A01822E912C9C01280D391D37FD6D
:1013D000C4C0803891050CF0C0C09B01200F311DA6
:1013E00037FDBBC0603471050CF0B7C0AB0177FFAF
:1013F00004C044275527461B570B477055279B01B0
:1014000077FF02C0295F3F4FE3E035952795EA95C6
:10141000E1F777FF08C02150310968E070E0DB0197
:10142000A41BB50BAD01602F66956695669570E0BF
:10143000077011F06F5F7F4FDB01A20FB31FBA83FC
:10144000A98339017694762C662477946794680E84
:10145000791EE12CF12C00E010E02301B0E84B0EE6
:10146000511C68E070E0DB01A41BB50BBC83AB83AF
:1014700069817A812617370709F46FC02830310552
:1014800009F46BC02F3FBFEF3B070CF45BC0B20108
:10149000600F711FDB01AF5ABE4FBE83AD83D80111
:1014A000A60DB71DAF5ABE4F6C0160E070E0681525
:1014B00079050CF047C0E0E8CE16D10409F442C02B
:1014C000D7FC34C02F3FFFEF3F0709F442C0FB01B8
:1014D000EE0DFF1DEA0DFB1DE491042E01C0EE0F81
:1014E0000A94EAF73C90E329EC9341155105F1F099
:1014F00027303105D9F0FB01EE0DFF1DEA0DFB1D74
:10150000E4912E2E312CF1010B8002C0F595E79568
:101510000A94E2F7F887EF83ED81FE813080EF8156
:10152000F885E3291F01ED81FE8120826F5F7F4FE7
:10153000ED81FE813196FE83ED83FFEFCF1ADF0A46
:101540001196B5CF2F5F3F4F00581F4FE80CF91C85
:101550008FCF4115510579F6E9CF28960FB6F8944B
:10156000DEBF0FBECDBFDF91CF911F910F91FF90D6
:10157000EF90DF90CF90BF90AF909F908F907F9033
:101580006F905F904F903F902F900895CF92DF9291
:10159000EF92FF920F931F93CF93DF937C0100E0B4
:1015A00010E06C012FEFC21AD20AE701F7FE0CC05F
:1015B000C0E0D0E009C0C817D90774F441E0BE010B
:1015C000C8010E94E40E2196C60121E4C216D1048E
:1015D00094F380E490E0EFCF0F5F1F4F00381105C8
:1015E00021F7DF91CF911F910F91FF90EF90DF9046
:1015F000CF9008958F929F92AF92BF920F931F93B7
:10160000CF93DF93CDB7DEB7A1970FB6F894DEBFC7
:101610000FBECDBF19A2423008F44AE08E010F5D23
:101620001F4F842E912CA12CB12CA50194010E9456
:10163000E214E62FB901CA0101501109EA3014F48D
:10164000E05D01C0E95CD801EC93232B242B252B12
:1016500061F70115110571F0F80101900020E9F71B
:101660003197AF01401B510BB80181E595E00E9415
:10167000FA0D02C080E090E0A1960FB6F894DEBFAC
:101680000FBECDBFDF91CF911F910F91BF90AF9053
:101690009F908F90089580E0E1E5F1E081118FEF58
:1016A000002481938193819381930394D1F70895CA
:1016B0001F920F920FB60F9211248F939F938091D8
:1016C000E1009091E100937F9093E10083FF0FC0D0
:1016D0001092E90091E09093EB001092EC0092E3FD
:1016E0009093ED001092500198E09093F00082FFEB
:1016F00020C093E09093E9009091F200992319F0B3
:101700009AE39093E80090916805992339F09091BD
:101710006805915090936805992389F190914F0144
:10172000992339F090914F01915090934F01992353
:1017300041F184FF10C08091E2008E7E8160809331
:10174000E2008091E1008F7E8093E10080914E0164
:101750008E7E806111C080FF16C08091E2008E7E77
:1017600080618093E2008091E1008E7E8093E100B1
:1017700080914E018E7E816080934E0104C05D9AFF
:10178000CDCF289AD6CF9F918F910F900FBE0F90FB
:101790001F9018951F920F920FB60F921124CF929F
:1017A000DF92EF92FF920F931F932F933F934F93EC
:1017B0005F936F937F938F939F93AF93BF93EF93B9
:1017C000FF93CF93DF93CDB7DEB76C97DEBFCDBF6E
:1017D0001092E9008091E80083FFEDC168E0CE013E
:1017E00045960E943E1082EF8093E8008D8987FF26
:1017F00005C09091E80090FFFCCF03C09EEF90934E
:10180000E800982F907609F0C6C09E892F89188D20
:1018100091110CC0803829F480914D018093F10022
:1018200002C01092F1001092F10048C1422F50E026
:10183000512B913051F4811141C14130510509F0D2
:101840003DC180914D018D7F0BC0933061F48111BA
:1018500035C14130510509F031C180914D0182609F
:1018600080934D012BC1953041F48091E80080FFB9
:10187000FCCF20682093E30021C1963009F05FC0BF
:10188000EB8CFC8C1092E90010924B0110924A01F3
:10189000123091F510924901109248010E945A09A4
:1018A00099E0BE016F5F7F4FDB01E92F1D92EA9542
:1018B000E9F799831A8391E09E8390EA98879AEFDB
:1018C000998720914A0130914B01275F3F4F3C831C
:1018D0002B838D831092E90010924B0110924A01E4
:1018E000F0924901E092480149E050E080E00E9416
:1018F00017100E945A09E2C0F0924901E092480193
:101900000E944008DC011296ED90FC901397E114C0
:10191000F10409F4C0C0D701ED91FC910480F58178
:10192000E02DBE016B5E7F4FC7010995009719F04E
:101930000CF0C4C0C7C0F701E084F184E8CF973051
:1019400009F4C0C0983021F481E08093F100B6C062
:10195000993009F0B3C0837009F0B4C0E3E1F1E05D
:1019600081E021E036E39081992361F08093E900E2
:101970002093EB0091919093EC003093ED008F5FFA
:10198000873089F78EE78093EA001092EA008F890A
:101990008093500193C08B8D9C8D1092E900109222
:1019A0004B0110924A019093490180934801898D1F
:1019B000811156C08E899D89913A59F4813209F07E
:1019C00081C047E050E06AE071E080E00E941710BB
:1019D00075C0913209F076C0833289F4888D90E029
:1019E000982F88272F89822BA0E0B0E080930601F2
:1019F00090930701A0930801B09309015FC0803262
:101A000069F48091E80082FFFCCF67E08AE091E012
:101A10000E943E108BEF8093E80006C0823209F0EE
:101A20004DC08F898093110180914C01882319F05A
:101A3000EEEFFAE002C0E0E0F8E080910A01909158
:101A40000B01A0910C01B0910D01803B9440A105C8
:101A5000B10509F07BC08091110180FF93C076C071
:101A60000E944008DC0112960D911C9113970115FC
:101A7000110541F1D801ED91FC910190F081E02D2B
:101A8000BE016B5E7F4FC8010995811117C0F80137
:101A900000851185ECCF113009F44EC0133091F45C
:101AA0008F89882309F445C0823081F440E860E1E1
:101AB0008AE99AE00E941914882321F08EEF80931E
:101AC000E80079C081E28093EB0075C0813029F491
:101AD00040E86BE08EE89AE0EDCF833099F70E9402
:101AE0004008DC011296ED90FC9013978E010F5F79
:101AF0001F4F6801E114F10479F0D701ED91FC91D9
:101B00000680F781E02DB801C7010995080F111D66
:101B1000F701E084F184EECFD8011C92F601019028
:101B20000020E9F73197BF016C197D0940E0C6013B
:101B3000C1CF68E77AE002C06CE77AE06115710511
:101B400009F2FB01449150E080E840CF0FB6F894D1
:101B5000A895809160008861809360001092600079
:101B60000FBEA895EE3F2AE0F20739F08091FE0AF9
:101B70009091FF0A91838083A1CF1092FF0A109267
:101B8000FE0A9CCFEE3F8AE0F80731F08081918118
:101B90009093FF0A8093FE0A87E797E791838083FB
:101BA0009BE088E10FB6F894A895809360000FBE83
:101BB0009093600083CF6C960FB6F894DEBF0FBE93
:101BC000CDBFDF91CF91FF91EF91BF91AF919F91E9
:101BD0008F917F916F915F914F913F912F911F91C5
:101BE0000F91FF90EF90DF90CF900F900FBE0F906E
:101BF0001F901895CF92DF92EF92FF920F931F9351
:101C0000CF93DF936C017A018B01C0E0D0E0CE1559
:101C1000DF0589F0D8016D918D01D601ED91FC9120
:101C20000190F081E02DC6010995892B11F47E0108
:101C300002C02196ECCFC701DF91CF911F910F9188
:101C4000FF90EF90DF90CF9008953FB7F894809188
:101C5000C6059091C705A091C805B091C90526B5E4
:101C6000A89B05C02F3F19F00196A11DB11D3FBFD4
:101C7000BA2FA92F982F8827820F911DA11DB11D62
:101C8000BC01CD0142E0660F771F881F991F4A955E
:101C9000D1F708950895089580E090E008950E9496
:101CA0000A158F929F92AF92BF92CF92DF92EF92DE
:101CB000FF926B017C010E94250E4B015C01C11457
:101CC000D104E104F104F1F00E94250EDC01CB0106
:101CD00088199909AA09BB09883E9340A105B10555
:101CE00070F321E0C21AD108E108F10888EE880EED
:101CF00083E0981EA11CB11CC114D104E104F104BD
:101D000019F7DDCFFF90EF90DF90CF90BF90AF90AD
:101D10009F908F9008951F920F920FB60F921124EB
:101D20002F933F938F939F93AF93BF9380914001E5
:101D300090914101A0914201B09143013091C505BC
:101D400023E0230F2D3720F40196A11DB11D05C0FE
:101D500026E8230F0296A11DB11D2093C50580938F
:101D6000400190934101A0934201B09343018091BF
:101D7000C6059091C705A091C805B091C905019607
:101D8000A11DB11D8093C6059093C705A093C805FA
:101D9000B093C905BF91AF919F918F913F912F91C2
:101DA0000F900FBE0F901F9018952D9A0895BC01AB
:101DB00080E090E00C94510E8FB18095807F669BFF
:101DC00088601C9B84600895EBEAFFE090E1969F99
:101DD000D001A0781124A80F6770E60FF11D94912F
:101DE000AF5ABE4F442319F08C91982B03C09095A5
:101DF0008C9198239C9308952F923F924F925F92DB
:101E00006F927F928F929F92AF92BF92CF92DF920A
:101E1000EF92FF920F931F93CF93DF93CDB7DEB76F
:101E200027970FB6F894DEBF0FBECDBFFC016A3016
:101E300069F425898189928938E0239F800D911D5D
:101E40001124928B818B108A1786A6C06D3009F4FD
:101E5000A3C09F838E8335882489298333893A835D
:101E600061887288E784F08880E8E816F104C4F09D
:101E7000AE81BF8155962C915597422F50E01F9609
:101E80008D919C915097B6E02B9F800D911D112450
:101E9000EE81FF81908B87872689211167C07CC0E6
:101EA000F0E46F16710424F7C70125E0329E800D1F
:101EB000911D112418161906DCF6432C512CC30170
:101EC00038E0339E800D911D11241816190684F6F2
:101ED00085E0689F800111240555154F20E0F80129
:101EE0002490253009F4212C430158E020FC02C045
:101EF000398101C03A8131110BC0F9818A81F8130F
:101F000007C026945150840C951C5111EFCF25C069
:101F100067018C2D8E198315A0F754018A2D88191D
:101F20008315B8F490E8C916D10478F4A0E4AA1691
:101F3000B10458F4432FB501C6012C833B835D8364
:101F40000E94E40E5D813B812C81BFEFAB1ABB0A7E
:101F5000E5CFEFEFCE1ADE0ADCCF2F5FE40CF51CE5
:101F60000F5F1F4F263009F0BACF82CF6AEF6403AC
:101F70009001659F300D112420583F4F28173907D5
:101F80005CF4AE81BF81ED91FC9111970190F081DD
:101F9000E02D6AE0CD01099581E090E027960FB62B
:101FA000F894DEBF0FBECDBFDF91CF911F910F918F
:101FB000FF90EF90DF90CF90BF90AF909F908F9069
:101FC0007F906F905F904F903F902F9008950C946A
:101FD000CC1440914A0150914B012091480130911D
:101FE000490142175307B4F49091E8009570E1F36A
:101FF0009091E80092FD19C08093F10080914A0110
:1020000090914B0101968F739927892B19F48EEFCC
:102010008093E80080914A0190914B010196909342
:102020004B0180934A0181E0089580E00895DF929A
:10203000EF92FF920F931F93CF93DF93D82E8A01D5
:102040007B01E40EF51EEB01CE15DF0571F0D7FE26
:1020500003C0FE01849101C088810E94E90F21968E
:102060008111F2CF8FEF9FEF01C0C801DF91CF91B7
:102070001F910F91FF90EF90DF900895615030F025
:102080002091F100FC0120830196F8CF289884E686
:1020900080934F010895789484B5826084BD84B59F
:1020A000816084BD85B5826085BD85B5816085BD53
:1020B00080916E00816080936E001092810080910B
:1020C0008100826080938100809181008160809393
:1020D00081008091800081608093800080919100D8
:1020E0008260809391008091910081608093910043
:1020F000809190008160809390008091C100846005
:102100008093C1008091C10082608093C100809162
:10211000C10081608093C1008091C3008160809381
:10212000C3008091C00082608093C0008091C20093
:1021300081608093C20080917A00846080937A00ED
:1021400080917A00826080937A0080917A00816029
:1021500080937A0080917A00806880937A00109250
:10216000500110924D0110924E018091D700816074
:102170008093D70080EA8093D80089B5806189BDBB
:1021800089B5826089BD09B400FEFDCF61E070E0D1
:1021900080E090E00E94510E8091D8008F7C806199
:1021A0008093D8008091E000807F8093E000809150
:1021B000E1008E7E8093E1008DE08093E200559AED
:1021C000209AEEEFFFE7859194918B3F9C4D19F497
:1021D00081E080934C0181EC80937C0085B1806F1D
:1021E00085B984B1877E84B984B1876E84B95E9ADB
:1021F0005F988AB1806D8AB9769A6E9881B3806F44
:1022000081BB899880B38D7080BB80E58CBD81E0F7
:102210008DBD85E090E00E94D70E5F9A85E090E04A
:102220000E94D70E5E985C98ECE5F1E08DE08E0F91
:1022300094919EBD00000DB407FEFDCF31968E1324
:10224000F7CF5C9A81E8809364008091650081609B
:102250008093650080E00E94B8090E94DC0E87FF31
:1022600024C05C9885EA8EBD00000DB407FEFDCF4A
:102270005C9A2E982F982D988091640080628093AC
:10228000640081E083BF889513BEFCCF2D980E9427
:10229000DC0E8478843871F00E94DC0E8471843105
:1022A00031F188EC90E00E94D70E0E94DC0E82FD96
:1022B000EDCF3AC00E94D50E88EC90E00E94D70E78
:1022C0002F9882E090E00E94CC148F3F29F06FEFAE
:1022D00082E090E00E94D41484EF91E00E94D70E37
:1022E0002F9A0E94DC0E84788438D9F3D5CF0E94CF
:1022F000D50E88EC90E00E94D70E2E9882E090E0F8
:102300000E94CC14882329F060E082E090E00E94D3
:10231000D41484EF91E00E94D70E2E9A0E94DC0E16
:1023200084718431D9F3BDCF0E94D50E82E090E054
:102330000E94CC14882331F03E9A3F9A81E080932A
:10234000440104C0109244013E983F9881E090E01F
:102350000E94E70F82FB112710F981FF3EC0111187
:102360002E98C0EFDFEF0E94DC0E86FF04C02E9A8D
:102370002F9A2D9A32C0112329F0C430D10511F4BF
:102380002E9A2F9881E00E94B80900E128E54CEAD6
:1023900050E0BE0184E190E00E94C70980E00E9405
:1023A000B8098FE090E00E94D70E2196C931D1057F
:1023B000D1F6112311F02F9A2D9880E991E00E9417
:1023C000D70E0E94D50EE0915505F091560501906B
:1023D000F081E02D85E595E0099582E390E00E948B
:1023E000D70E0E94DC0E8111F8CF0E944B0B109289
:1023F000630510926205109261051092600581E2FA
:1024000080935C0520E0422E20E0522E38E0E32E3F
:10241000F12C48E3C42ED12CC0E1D0E058E1A52E28
:10242000B12C60E2862E912C7AE2672E712C11E09D
:1024300085E1382E98E6292E8FB7F8944091400117
:102440005091410160914201709143018FBF809191
:102450005D05942F981B892F90915E05992329F093
:1024600080935F0510925E05DDC190915C05891730
:1024700040F48F5F891708F0D5C113BF889513BE4C
:10248000D1C110935E0540935D05809158059091F0
:1024900059050196909359058093580580915A05E6
:1024A00080935B050E94DC0E80935A050E944B0BC3
:1024B00010926305109262051092610510926005FA
:1024C00080910501823009F463C028F4882361F00B
:1024D000813099F1A4C1843009F4B0C008F483C0FC
:1024E000853009F472C19BC188E00E948C0981117A
:1024F00010930501F0926105E0926005D0926305AA
:10250000C092620582E29AE00E949709D093610529
:10251000C0936005B0926305A092620583E19AE0E2
:102520000E949709D0936105C0936005909263055E
:102530008092620584E09AE070C188E00E948C0974
:10254000882319F084E080930501F0926105E09200
:102550006005D0926305C092620584EF99E00E9405
:102560009709D0936105C0936005B0926305A0926E
:1025700062058BEE99E00E949709D0936105C093A4
:102580006005909263058092620580EE99E045C1F6
:1025900088E00E948C09882319F023E0209305012C
:1025A000F0926105E0926005D0926305C0926205E9
:1025B0008CEC99E00E949709D0936105C093600567
:1025C000B0926305A09262058DEB99E00E94970995
:1025D000D0936105C0936005909263058092620577
:1025E0008FEA99E01AC188E00E948C09882319F0CB
:1025F00084E080930501F0926105E0926005D0923D
:102600006305C092620588E999E00E949709D0931A
:102610006105C0936005B0926305A092620589E8E8
:1026200099E00E949709D0936105C093600590924C
:102630006305809262058BE799E0EFC080914701C6
:10264000813069F130F08230F1F1843009F451C009
:102650006CC080914601811103C01093460102C0F5
:102660001092460180E80E948C09882341F0109264
:10267000460110924501309202011093470180E11A
:102680000E948C09882309F450C0109246011092D0
:1026900045011093020182E08093470146C080917A
:1026A0004501853020F48F5F8093450106C010926C
:1026B00047011092460110920201809101018D3074
:1026C000A0F1825013C080914501853020F48F5FC6
:1026D0008093450106C01092470110924601109266
:1026E000020180910101843200F58E5F8093010127
:1026F0001CC00E94DC0E85FF0AC080910001882367
:1027000021F081508093000102C0109200010E94CC
:10271000DC0E86FF0AC080910001883620F48F5FAE
:102720008093000102C0209200010E944B0B109286
:102730006305109262057092610560926005609178
:10274000460170E080E090E04AE00E94FA0A1092B0
:102750006105109260051092630510926205E09188
:102760004601F0E0EE5FFE4F608170E080E090E0B7
:102770004AE00E94FA0A8FE390E00E94C60A83E3CF
:1027800090E00E94C60A87E290E00E94C60A8BE1B0
:1027900090E00E94C60AE0914601F0E0EE5FFE4F35
:1027A000408198E4949FA001112445565E4F6091AA
:1027B000010170E08091000108E128E190E00E94B1
:1027C000C70980E00E94B8092AC088E00E948C09ED
:1027D000811110920501F0926105E0926005D0929E
:1027E0006305C092620586E891E00E949709D09344
:1027F0006105C0936005B0926305A092620587E70A
:1028000091E00E949709D0936105C0936005909272
:1028100063058092620589E691E00E94970980E055
:102820000E94B8094114510409F406CE0E94000028
:10283000FECDCF92DF92EF92FF920F931F93CF9333
:10284000DF931F92CDB7DEB7182F062FE42E862F09
:10285000880F8E5F99830E94E90F83E00E94E90F41
:10286000F12EC12E9981D92E8C2D8F19801798F4B5
:10287000F601E7FE02C0849101C080810E94E90F49
:10288000182F80E00E94E90F8123FFEFCF1ADF0AA3
:102890008111EACF01C081E00F90DF91CF911F91AC
:1028A0000F91FF90EF90DF90CF900895E5E7F5E06E
:1028B0001382128288EE93E0A0E0B0E084839583D7
:1028C000A683B7838DE191E0918380838FEF9FEFA3
:1028D00095878487E1E5F5E01382128211861286DE
:1028E00080E183871086178215868FE291E09183BD
:1028F00080838DE391E095838483108A1786128A02
:10290000118A81E0838B148A858B168A08950F9330
:102910001F93CF93DF938C0181E090E00E94E70F3B
:1029200080FF32C08AE090E00E94E70F9FEF980F8F
:102930009E3F50F522E330E0D80150963C932E9311
:102940001F9728E330E052963C932E935197CBE0AB
:10295000D0E0D801ED91FC910190F081E02D682F3D
:10296000C8010995CE010E94E70F2196C131D1051A
:1029700081F780E00E94B80988EE93E0DF91CF9163
:102980001F910F910C94D70EDF91CF911F910F9152
:10299000089504970C948714F999FECF92BD81BDD8
:1029A000F89A992780B50895262FF999FECF1FBA76
:1029B00092BD81BD20BD0FB6F894FA9AF99A0FBE68
:1029C00001960895A1E21A2EAA1BBB1BFD010DC0A2
:1029D000AA1FBB1FEE1FFF1FA217B307E407F507CF
:1029E00020F0A21BB30BE40BF50B661F771F881FAB
:1029F000991F1A9469F760957095809590959B0141
:102A0000AC01BD01CF010895EE0FFF1F0590F491B9
:102A1000E02D099481E090E0F8940C940F15F8945F
:022A2000FFCFE6
:102A22000C1800070E01FFFFFFFF00E1000000008D
:102A3200000000C18081000000000000005408D5A1
:102A42000875086A08BB087908970800000000FCAE
:102A52000EFA0D4C0E4B0E8714FCFF0000C9140039
:00000001FF
